:020000040000FA
:06000000C5EF1FF0120025
:06080000C5EF1FF012001D
:060808007CEF1EF012005F
:060818008AEF1EF0120041
:02082A000000CC
:04082C0000000000C8
:10083000000000000000000012001E0EE66E79ECC1
:100840001FF0E5521200060EE66E79EC1FF0E5523D
:1008500012000C0EE66EA6EC1FF0E5521200D9CF86
:10086000E6FFE1CFD9FF0101A65110E0E8EC1FF04F
:10087000FC0EDBCFE6FFFD0EDBCFE6FFFE0EDBCF8F
:10088000E6FFA2EC1EF0E552E552E552E552E7CF55
:10089000D9FF1200D9CFE6FFE1CFD9FFFE0EDBCFA3
:1008A000F3FFDB06F350000918E044EC1FF00009E9
:1008B000FCE1500E0101A55DF1E2EBEC1EF0E66EED
:1008C0000101A551A52BEA6A550FE96E010EEA2236
:1008D000E552E750EF6EE2E1E1D7E552E7CFD9FF0D
:1008E0001200D9CFE6FFE1CFD9FFFD0EDB50F36E4A
:1008F000FE0EDBCFF4FFF350F45C1FE2E8EC1FF0D8
:10090000500E0101A55DF1E2FE0EDBCFF3FFDB2A05
:10091000F350E66EE66A29EC1FF0E552E552E66E0A
:100920000101A551A52BEA6A550FE96E010EEA22D5
:10093000E552E750EF6ED9E1D8D7E552E7CFD9FFBE
:100940001200806A0F0EC16E070EB46EF19E939076
:100950009290809081909282928492869288928ADC
:10096000949094929494949C949E82908292829477
:10097000829C829E0101A66B546BF16B0F0EBE6FC1
:10098000A96B010EAA6F506B516BA56B970EE66EAB
:100990000DEC1FF0E552E0EF1CF02B0EE66EEBECD9
:1009A0001CF0E5521200D9CFE6FFE1CFD9FF030ECC
:1009B000E1260101A9510BE0AB0509E16D96010E9D
:1009C000AA6FA751FEE0F29E31EC16F0F2D3030EAF
:1009D0000101FC5D03E36D50020B1FE0030EFC5DA3
:1009E00003E16D50020B19E10101AA5101E0E1D3CD
:1009F0008090829082928294829C829EBE9544ECEA
:100A00001FF00009FCE1BEC1E6FF56EC1EF0E55206
:100A1000F29E0101010EAA6FCCD30101AA5101E19E
:100A200014D1E8EC1FF0000EE66EE66A29EC1FF028
:100A3000E552E5520F0B0101BE6F010EE66EE66A4C
:100A400029EC1FF0E552E5520101AB6FAC0EE66EEA
:100A5000010EE66E020EE66EE66A29EC1FF0E55224
:100A6000E552E66EF8EC12F0E552E552E552B50EAD
:100A7000E66E010EE66E030EE66EE66A29EC1FF0E6
:100A8000E552E552006E016AFF0ED8800056000E56
:100A90000156020E416E426A00C03CF001C03DF0BA
:100AA0000AEC1EF03CC000F03DC001F03C50E66E88
:100AB000F8EC12F0E552E552E552DF6A050EDF5C14
:100AC00037E2E8EC1FF0DF50090DF3CF00F0F4CF70
:100AD00001F0BF0E0026010E012200C0E6FF01C09A
:100AE000E6FF090EDF24E66EE66A29EC1FF0E55208
:100AF000E552E66EF8EC12F0E552E552E552040ECE
:100B0000DF24E66EE66A29EC1FF0E552E5520008A4
:100B100002E3000E01D0010EE66EDF50EA6AEC0F30
:100B2000E96E010EEA22E552E750EF6EDF2AC6D7E2
:100B300044EC1FF00009FCE1BEC1E6FF56EC1EF0DC
:100B4000E552DF6A080EDF5C3AE244EC1FF0000970
:100B5000FCE1080EDF02F350400FE66E56EC1EF08B
:100B6000E552080EDF02F350100FE76E020EE7CFDA
:100B7000DBFF010EDB6A080EF36E010EDBCFF4FF24
:100B8000F350F45C1AE2E8EC1FF044EC1FF00009AB
:100B9000FCE1010EDBCFE6FF020EDB50E552E7245D
:100BA000E66EE66A29EC1FF0E552E552E66E30EC9F
:100BB0001EF0E552010EDB2ADED7DF2AC3D7DF6A3B
:100BC000040EDF5C3AE244EC1FF00009FCE1DF2890
:100BD000E66E010EE66E4CEC11F0E552E552140E95
:100BE000DF02F350500FE76E020EE7CFDBFF010E7E
:100BF000DB6A140EF36E010EDBCFF4FFF350F45CEE
:100C00001AE2E8EC1FF044EC1FF00009FCE1010ED1
:100C1000DBCFE6FF020EDB50E552E724E66EE66A24
:100C200029EC1FF0E552E552E66E30EC1EF0E5527D
:100C3000010EDB2ADED7DF2AC3D70101FA0EA86F27
:100C4000AB5102E0A76BF28EAA6BB42BB251030D2D
:100C5000F3CFE9FFF4CFEAFFAC0EE926010EEA225A
:100C6000020EE926000EEA22EF50B45D0AE3AC0E54
:100C7000E66E010EE66E90EC12F0E552E5520009C8
:100C80000FE00101B251030DF3CFE9FFF4CFEAFF0A
:100C9000AC0EE926010EEA22EE52EF50B45D02E3FB
:100CA000000E01D0010EE8B08080E8A08090010124
:100CB000BD2BBB51030DF3CFE9FFF4CFEAFFB50E17
:100CC000E926010EEA22020EE926000EEA22EF5082
:100CD000BD5D0AE3B50EE66E010EE66E90EC12F015
:100CE000E552E55200090FE00101BB51030DF3CFBE
:100CF000E9FFF4CFEAFFB50EE926010EEA22EE5233
:100D0000EF50BD5D02E3000E01D0010EE8B081801E
:100D1000E8A081900101EC5132E0C72BC551030DD1
:100D2000F3CFE9FFF4CFEAFFBF0EE926010EEA2276
:100D3000020EE926000EEA22EF50C75D0AE3BF0E5D
:100D4000E66E010EE66E90EC12F0E552E5520009F7
:100D50000FE00101C551030DF3CFE9FFF4CFEAFF26
:100D6000BF0EE926010EEA22EE52EF50C75D02E304
:100D7000000E01D0010EE8B08280E8A0829001014F
:100D8000ED5132E0D02BCE51030DF3CFE9FFF4CF7C
:100D9000EAFFC80EE926010EEA22020EE926000E3D
:100DA000EA22EF50D05D0AE3C80EE66E010EE66E51
:100DB00090EC12F0E552E55200090FE00101CE512E
:100DC000030DF3CFE9FFF4CFEAFFC80EE926010EC9
:100DD000EA22EE52EF50D05D02E3000E01D0010E88
:100DE000E8B08282E8A082920101EE5132E0D92B74
:100DF000D751030DF3CFE9FFF4CFEAFFD10EE92677
:100E0000010EEA22020EE926000EEA22EF50D95D19
:100E10000AE3D10EE66E010EE66E90EC12F0E5529A
:100E2000E55200090FE00101D751030DF3CFE9FFAF
:100E3000F4CFEAFFD10EE926010EEA22EE52EF507E
:100E4000D95D02E3000E01D0010EE8B08284E8A073
:100E500082940101EF5132E0E22BE051030DF3CF18
:100E6000E9FFF4CFEAFFDA0EE926010EEA22020ECC
:100E7000E926000EEA22EF50E25D0AE3DA0EE66EA2
:100E8000010EE66E90EC12F0E552E55200090FE01B
:100E90000101E051030DF3CFE9FFF4CFEAFFDA0ED1
:100EA000E926010EEA22EE52EF50E25D02E3000E67
:100EB00001D0010EE8B0828CE8A0829C0101F051C3
:100EC00032E0EB2BE951030DF3CFE9FFF4CFEAFF5A
:100ED000E30EE926010EEA22020EE926000EEA22BE
:100EE000EF50EB5D0AE3E30EE66E010EE66E90EC6A
:100EF00012F0E552E55200090FE00101E951030D3E
:100F0000F3CFE9FFF4CFEAFFE30EE926010EEA2270
:100F1000EE52EF50EB5D02E3000E01D0010EE8B09F
:100F2000828EE8A0829E0101A9511EE0A75100080F
:100F300001E33FD1A76B44EC1FF00009FCE1010E77
:100F4000E66E0E0EE66E4CEC11F0E552E55244EC06
:100F50001FF00009FCE10101AB07300EAB25E66E86
:100F600030EC1EF0E55225D12B0EA75D12E3A76BE6
:100F7000AB050BE1BE9544EC1FF00009FCE1BEC1DE
:100F8000E6FF56EC1EF0E552F29E0101AB5101E086
:100F9000AB07060E0101FC5D01E20BD10101A82B9C
:100FA000A851190801E3ECD0F151020B14E1805073
:100FB000020B11E1F183500EA55D22E2A551A52B94
:100FC000EA6A550FE96E010EEA22410EEF6E000942
:100FD00017E0010E18D0F151020B15E08050020B02
:100FE00012E0F193500EA55D0BE2A551A52BEA6A24
:100FF000550FE96E010EEA22610EEF6E000902E163
:10100000000E01D0010EF151040B14E18050040BCD
:1010100011E1F185500EA55D22E2A551A52BEA6AEA
:10102000550FE96E010EEA22420EEF6E000917E03D
:10103000010E18D0F151040B15E08050040B12E0A2
:10104000F195500EA55D0BE2A551A52BEA6A550F4F
:10105000E96E010EEA22620EEF6E000902E1000E57
:1010600001D0010EF151080B14E18050080B11E181
:10107000F187500EA55D22E2A551A52BEA6A550F16
:10108000E96E010EEA22430EEF6E000917E0010E31
:1010900018D0F151080B15E08050080B12E0F197C1
:1010A000500EA55D0BE2A551A52BEA6A550FE96E1E
:1010B000010EEA22630EEF6E000902E1000E01D07C
:1010C000010EF151100B14E18050100B11E1F18968
:1010D000500EA55D22E2A551A52BEA6A550FE96ED7
:1010E000010EEA22440EEF6E000917E0010E18D03F
:1010F000F151100B15E08050100B12E0F199500ED9
:10110000A55D0BE2A551A52BEA6A550FE96E010E0C
:10111000EA22640EEF6E000902E1000E01D0010E1A
:10112000F151200B14E18050200B11E1F18B500E96
:10113000A55D22E2A551A52BEA6A550FE96E010EC5
:10114000EA22450EEF6E000917E0010E18D0F151AA
:10115000200B15E08050200B12E0F19B500EA55D96
:101160000BE2A551A52BEA6A550FE96E010EEA22A2
:10117000650EEF6E000902E1000E01D0010EA86BB2
:10118000000161510EE10001550E626F010E636FA7
:10119000A5C166F00001676B0001010E616F0101DE
:1011A000A56B44EC1FF0000904E10DD8000901E033
:1011B0002BD8030EE15C02E2E16AE552E16EE552F2
:1011C000E7CFD9FF120001015051D880515512E3E9
:1011D000500EE66E000EE66E010EE66E79EC19F02A
:1011E000E552E552E552000901E1000C60C051F101
:1011F0000101506B5051502BEA6A000FE96E010E4D
:10120000EA22EFCF52F1010C010154513D0A02E1F3
:1012100059EF0DF0010A02E149EF0DF00B0A02E16E
:101220002BEF0DF0010A01E1F6D3020A01E1B4D27D
:10123000070A01E198D2060A01E185D2070A01E115
:1012400075D2110A01E160D2010A01E159D2030A03
:1012500001E14FD2010A01E148D2040A01E130D292
:101260003B0A01E114D22F0A01E102D21F0A01E177
:10127000EBD1010A01E1D4D1030A01E1BDD1010A98
:1012800001E1A6D1070A01E18FD1010A01E178D17C
:10129000030A01E162D1010A01E15BD1360A01E1F1
:1012A00051D1030A01E1CDD0060A01E1B0D0010A13
:1012B00001E1A9D0020A01E19BD0010A01E18ED02F
:1012C0000E0A65E0010A5BE0030A40E0180A32E01A
:1012D000010A24E0070A18E0010A12E00B0A0EE0F6
:1012E000010A01E01200FE0E525D02E1010EDFD3A1
:1012F00052C1E6FF30EC1EF0E552120068EF0DF02F
:1013000052C153F10B0ED3D352C1E6FF53C1E6FFD6
:101310004CEC11F0E552E5520101B9D3080E52032D
:10132000F350400FE66E56EC1EF0E5520101536B90
:101330000D0EBDD352C1E6FF30EC1EF0E5520101A7
:10134000532B080E535D01E2C2D3A1D352C1ABF1BE
:1013500052C1E6FF010EE66EE66A2FEC04F0E5529C
:10136000E552E5520101A76BAB5102E0010E01D03D
:10137000000EE8B0F28EE8B08AD3F29E88D352C154
:10138000E6FF020EE66EE66A2FEC04F089D152C148
:10139000E6FF030EE66EE66A2FEC04F0E552E55236
:1013A000E552B50EE66E010EE66E01015251006E79
:1013B000016AFF0ED8800056000E0156020E416EE3
:1013C000426A00C03CF001C03DF00AEC1EF03CC097
:1013D00000F03DC001F03C50E66E6BD15205536FFA
:1013E000E850EA6AEC0FE96E010EEA22EF6A24D0B7
:1013F0005205536FE850EA6AEC0FE96E010EEA22DB
:10140000010EEF6E19D05205536F1B0E50D353517E
:10141000090DF3CF00F0F4CF01F0BF0E0026010E4E
:10142000012200C0E6FF01C0E6FF52C1E6FFF8EC72
:1014300012F0E552E552E55253C1E6FF6DEC11F0B2
:101440003CD1520517E1500EA55D01E377D08050E5
:10145000020B02E1410E01D0610EE66EA551A52BF3
:10146000EA6A550FE96E010EEA22E552E750EF6E87
:1014700067E164D0020E525D16E1500EA55D5EE29A
:101480008050040B02E1420E01D0620EE66EA551BF
:10149000A52BEA6A550FE96E010EEA22E552E750E4
:1014A000EF6E4EE14BD0030E525D16E1500EA55D7E
:1014B00045E28050080B02E1430E01D0630EE66E58
:1014C000A551A52BEA6A550FE96E010EEA22E552F5
:1014D000E750EF6E35E132D0040E525D16E1500E4A
:1014E000A55D2CE28050100B02E1440E01D0640E89
:1014F000E66EA551A52BEA6A550FE96E010EEA22A8
:10150000E552E750EF6E1AE01BD0050E525D01E088
:10151000BED2500EA55D12E28050200B02E1450EB6
:1015200001D0650EE66EA551A52BEA6A550FE96E4E
:10153000010EEA22E552E750EF6E02E1000EA7D25B
:10154000010EA5D2520502E0000E01D0010EA66FD9
:101550009ED252C153F1290EAAD2E8EC1FF052C11B
:10156000E6FF080E01015303F350100FE66EE66A22
:10157000A2EC1EF0E552E552E55201012A0E97D287
:10158000E8EC1FF052C1E6FF080E01015303F350CF
:10159000100F010FE66EE66AA2EC1EF0E552E5526E
:1015A000E55201012B0E83D2E8EC1FF052C1E6FF99
:1015B000080E01015303F350100F020FE66EE66AA6
:1015C000A2EC1EF0E552E552E55201012C0E6FD25D
:1015D000E8EC1FF052C1E6FF080E01015303F3507F
:1015E000100F030FE66EE66AA2EC1EF0E552E5521C
:1015F000E55201012D0E5BD2E8EC1FF052C1E6FF6F
:10160000080E01015303F350100F040FE66EE66A53
:10161000A2EC1EF0E552E552E55201012E0E47D232
:10162000E8EC1FF052C1E6FF080E01015303F3502E
:10163000100F050FE66EE66AA2EC1EF0E552E552C9
:10164000E55201012F0E33D2E8EC1FF052C1E6FF44
:10165000080E01015303F350100F060FE66EE66A01
:10166000A2EC1EF0E552E552E5520101300E1FD208
:10167000E8EC1FF052C1E6FF080E01015303F350DE
:10168000100F070FE66EE66AA2EC1EF014D0E8EC2D
:101690001FF052C1E6FF020EE66EE66AA2EC1EF0F3
:1016A000E552E552E552AC0EE66E010EE66E52C111
:1016B000E6FFF8EC12F0E552E552E5520101E7D100
:1016C000E8EC1FF052C1E6FF500E01015325E66E13
:1016D000E66AA2EC1EF0E552E552E5520101532BF9
:1016E000500E535D01E2F3D1D2D15205536F210E5A
:1016F000DED1E8EC1FF052C1E6FF090E01010FD068
:101700005205536F230ED3D1E8EC1FF00101525163
:10171000000802E3000E01D0010EE66E040E532510
:10172000E66EE66AA2EC1EF0E55219D0080E5203EE
:10173000F350400FE66E56EC1EF0E552080EE66ED2
:101740004AEC04F00DD0080E5203F350100F526F04
:10175000080E5225E66E52C1E6FF71EC04F0E55228
:10176000E552010194D1500EA55D01E38DD15205E2
:10177000EA6AEC0FE96E010EEA22EF50E66EA5511F
:10178000A52BEA6A550FE96E010EEA22E552E750F1
:10179000EF6E01E05ED178D1500EA55D01E374D10A
:1017A0005205090DF3CFE9FFF4CFEAFFBF0EE9269A
:1017B000010EEA22020EE926000EEA22EFCF24F003
:1017C000256A266A276A5205090DF3CFE9FFF4CF8F
:1017D000EAFFBF0EE926010EEA22EFCF20F0216AD0
:1017E000226A236A20C03AF021C03BF022C03CF0BC
:1017F00023C03DF024C03FF025C040F026C041F09A
:1018000027C042F0D2EC1DF036C01CF037C01DF0EE
:1018100038C01EF039C01FF001015205090DF3CF89
:10182000E9FFF4CFEAFFBF0EE926010EEA22030E1C
:10183000E926000EEA22020EE926000EEA22EFCF88
:101840002CF02D6A2E6A2F6A5205090DF3CFE9FF9D
:10185000F4CFEAFFBF0EE926010EEA22030EE926C5
:10186000000EEA22EFCF28F0296A2A6A2B6A28C0E4
:101870003AF029C03BF02AC03CF02BC03DF02CC010
:101880003FF02DC040F02EC041F02FC042F0D2EC0E
:101890001DF01C503624186E1D503720196E1E5036
:1018A00038201A6E1F5039201B6E01015205090D98
:1018B000F3CFE9FFF4CFEAFFBF0EE926010EEA22DB
:1018C000EE52EFCF0CF00D6A0E6A0F6A5205090D49
:1018D000F3CFE9FFF4CFEAFFBF0EE926010EEA22BB
:1018E000EFCF08F0096A0A6A0B6A08C03AF009C02B
:1018F0003BF00AC03CF00BC03DF00CC03FF00DC007
:1019000040F00EC041F00FC042F0D2EC1DF036C0E6
:1019100004F037C005F038C006F039C007F0010107
:101920005205090DF3CFE9FFF4CFEAFFBF0EE92618
:10193000010EEA22030EE926000EEA22EE52EFCF54
:1019400014F0156A166A176A5205090DF3CFE9FFFC
:10195000F4CFEAFFBF0EE926010EEA22030EE926C4
:10196000000EEA22EFCF10F0116A126A136A10C05B
:101970003AF011C03BF012C03CF013C03DF014C06F
:101980003FF015C040F016C041F017C042F0D2EC55
:101990001DF004503624006E05503720016E0650AD
:1019A0003820026E07503920036E3F68406A416A52
:1019B000426A00C03AF001C03BF002C03CF03D6E0C
:1019C000D2EC1DF036C000F037C001F038C002F094
:1019D00039C003F036C03AF037C03BF038C03CF0B5
:1019E00039C03DF018C03FF019C040F01AC041F0B6
:1019F0001BC042F0C7EC1EF03A50E66E0101A55143
:101A0000A52BEA6A550FE96E010EEA22E552E7506E
:101A1000EF6E1FE139D0500EA55D36E2040E52255F
:101A2000FF0FE66EE66A29EC1FF0E552E55200086A
:101A300002E3000E01D0010EE66E0101A551A52BB7
:101A4000EA6A550FE96E010EEA22E552E750EF6EA1
:101A50001BE0010E1CD0500EA55D16E2090E5225AA
:101A6000FF0FE66EE66A29EC1FF0E552E552E66EDE
:101A70000101A551A52BEA6A550FE96E010EEA2274
:101A8000E552E750EF6E02E1000E01D0010E546BFB
:101A90001200E8EC1FF052C1E6FF0E0EE66EE66A99
:101AA000A2EC1EF0E552E552E55201013D0E546FE5
:101AB0001200E8EC1FF052C1E6FF0F0EE66EE66A78
:101AC000A2EC1EF0E552E552E5520101546B120002
:101AD00001015251010A01E1DAD3FF0A01E1D2D337
:101AE000EA0A01E1CCD3070A01E1C7D3010A01E107
:101AF000B9D3030A01E1B4D3010A01E193D31F0A68
:101B000001E175D3010A01E157D3030A01E139D399
:101B1000070A01E134D3030A01E12FD3010A01E1ED
:101B2000F1D20F0A01E1ECD2010A01E116D2030A57
:101B300001E131D1010A01E11DD1070A01E109D119
:101B4000340A01E1F5D0010A01E1E1D0030A01E123
:101B5000A7D0010A01E1A2D0F50A01E19DD0810AD6
:101B600001E197D0820A01E192D0510A01E18DD0C2
:101B7000570A01E188D0070A01E183D0030A01E195
:101B80007ED0A60A01E17BD0310A01E176D0010ABC
:101B900072E0180A6EE0DF0A6AE0C80A66E0C10A6D
:101BA00064E0C80A60E0170A5CE00A0A55E0010A2E
:101BB00051E0040A4DE0100A49E00C0A39E0070A36
:101BC00035E0180A31E0010A2DE00C0A16E0040A9B
:101BD00001E060D3BE85BEC1E6FF000EE66EE66A98
:101BE0002FEC04F0E552E552E552BEC1E6FF56EC9B
:101BF0001EF0E5520101150E43D3BE95BEC1E6FFAE
:101C0000000EE66EE66A2FEC04F0E552E552E5526E
:101C1000BEC1E6FF56EC1EF0E5520101546BAB6B02
:101C2000F29E1200BE8305D0BE9303D0BE8101D0C8
:101C3000BE91BEC1E6FF000EE66EE66A2FEC04F030
:101C4000E552E552E552BEC1E6FF08D0010E05D0CF
:101C5000020E03D0100E01D0140EE66E56EC1EF0EC
:101C60000AD30A0E0DD3170E0BD3160E09D31F0E6F
:101C700007D30C0E05D3190E03D3180E01D31A0E79
:101C8000FFD2200EFDD2220EFBD21E0EF9D2280E5C
:101C9000F7D2536B240EF4D21D0EF2D23C0EF0D2CA
:101CA000E8EC1FF0500E0101A55D14E20E0EE66E89
:101CB000E66A29EC1FF0E552E552E66E0101A551F6
:101CC000A52BEA6A550FE96E010EEA22E552E750AC
:101CD000EF6E02E1000E01D0010E500EA55D01E392
:101CE000BBD20F0EE66EE66A29EC1FF0E552E55214
:101CF000E66E0101A551A52BEA6A550FE96E010EAA
:101D0000EA22E552E750EF6E01E0A8D2A5D2500ECC
:101D1000A55D01E3A1D2A551A52BEA6A550FE96E95
:101D2000010EEA22120EEF6E000901E097D294D262
:101D3000500EA55D01E390D2A551A52BEA6A550F7F
:101D4000E96E010EEA225B0EEF6E000901E086D219
:101D500083D2500EA55D01E37FD2A551A52BEA6A7F
:101D6000550FE96E010EEA22BEC1EFFFEF5001E010
:101D700075D272D2500EA55D01E36ED2A551A52B8E
:101D8000EA6A550FE96E010EEA22ABC1EFFFEF5090
:101D900001E064D261D2500EA55D01E35DD2B7C10E
:101DA00028F0296A2A6A2B6AB5C124F0256A266AB6
:101DB000276AB5C13AF025C03BF026C03CF027C0E9
:101DC0003DF0B7C13FF029C040F02AC041F02BC020
:101DD00042F0D2EC1DF036C020F037C021F038C000
:101DE00022F039C023F0BAC130F0316A326A336A66
:101DF000B8C12CF02D6A2E6A2F6AB8C13AF02DC0F6
:101E00003BF02EC03CF02FC03DF0BAC13FF031C0D6
:101E100040F032C041F033C042F0D2EC1DF020500F
:101E200036241C6E215037201D6E225038201E6E25
:101E3000235039201F6EB6C110F0116A126A136A5E
:101E4000B5C10CF00D6A0E6A0F6AB5C13AF00DC04B
:101E50003BF00EC03CF00FC03DF0B6C13FF011C0EA
:101E600040F012C041F013C042F0D2EC1DF036C079
:101E700008F037C009F038C00AF039C00BF0B9C11A
:101E800018F0196A1A6A1B6AB8C114F0156A166A42
:101E9000176AB8C13AF015C03BF016C03CF017C045
:101EA0003DF0B9C13FF019C040F01AC041F01BC06D
:101EB00042F0D2EC1DF008503624046E0950372051
:101EC000056E0A503820066E0B503920076E3F68A9
:101ED000406A416A426A04C03AF005C03BF006C05D
:101EE0003CF03D6ED2EC1DF036C004F037C005F07A
:101EF00038C006F039C007F036C03AF037C03BF0C2
:101F000038C03CF039C03DF01CC03FF01DC040F06F
:101F10001EC041F01FC042F0C7EC1EF03AC000F0F6
:101F20003BC001F03CC002F03DC003F0D890003649
:101F3000013602360336001E011E021E031E010179
:101F4000A551A52BEA6A550FE96E010EEA2200C0E1
:101F5000EFFFEF5001E082D17FD1500EA55D01E38C
:101F60007BD1AEC124F0256A266A276AACC120F075
:101F7000216A226A236AACC13AF021C03BF022C038
:101F80003CF023C03DF0AEC13FF025C040F026C07C
:101F900041F027C042F0D2EC1DF036C01CF037C033
:101FA0001DF038C01EF039C01FF0B1C12CF02D6AF1
:101FB0002E6A2F6AAFC128F0296A2A6A2B6AAFC13C
:101FC0003AF029C03BF02AC03CF02BC03DF0B1C133
:101FD0003FF02DC040F02EC041F02FC042F0D2ECB7
:101FE0001DF01C503624186E1D503720196E1E50DF
:101FF00038201A6E1F5039201B6EADC10CF00D6ACF
:102000000E6A0F6AACC108F0096A0A6A0B6AACC1B1
:102010003AF009C03BF00AC03CF00BC03DF0ADC146
:102020003FF00DC040F00EC041F00FC042F0D2ECC6
:102030001DF036C004F037C005F038C006F039C0D6
:1020400007F0B0C114F0156A166A176AAFC110F034
:10205000116A126A136AAFC13AF011C03BF012C0A4
:102060003CF013C03DF0B0C13FF015C040F016C0C9
:1020700041F017C042F0D2EC1DF004503624006E3F
:1020800005503720016E06503820026E0750392067
:10209000036E3F68406A416A426A00C03AF001C07C
:1020A0003BF002C03CF03D6ED2EC1DF036C000F0BB
:1020B00037C001F038C002F039C003F036C03AF042
:1020C00037C03BF038C03CF039C03DF018C03FF09D
:1020D00019C040F01AC041F01BC042F0C7EC1EF01E
:1020E0003A50E66E0101A551A52BEA6A550FE96E3B
:1020F000010EEA22E552E750EF6E01E0AFD0ACD01E
:10210000320EBED0010EE66EE66EC6D8E552E5523E
:10211000140EE66E4AEC04F0E55244EC1FF00009A0
:10212000FCE1020EE66E010EE66EB6D8E552E5520F
:10213000140EE66E4AEC04F0E55244EC1FF0000980
:10214000FCE1030EE66E010EE66EA6D8E552E552FE
:10215000140EE66E4AEC04F0E55244EC1FF0000960
:10216000FCE1040EE66E010EE66E96D8E552E552ED
:10217000140EE66E4AEC04F07ED0330E81D0340E9D
:102180007FD0E8EC1FF0500E0101A55D65E2000E66
:10219000E66EE66A29EC1FF0E552E552E66E0101B3
:1021A000A551A52BEA6A550FE96E010EEA22E55208
:1021B000E750EF6E53E150D0E8EC1FF0500E0101F4
:1021C000A55D4AE2010EE66EE66A29EC1FF0E552D3
:1021D000E552E66E0101A551A52BEA6A550FE96E9D
:1021E000010EEA22E552E750EF6E38E135D0E8EC17
:1021F0001FF0500E0101A55D2FE2030EE66EE66AA8
:1022000029EC1FF0E552E552E66E0101A551A52B20
:10221000EA6A550FE96E010EEA22E552E750EF6EC9
:102220001DE11AD0E8EC1FF0500E0101A55D14E28B
:10223000020EE66EE66A29EC1FF0E552E552E66E04
:102240000101A551A52BEA6A550FE96E010EEA229C
:10225000E552E750EF6E02E1000E1CD0010E1AD0DD
:10226000350E0ED0E8EC1FF0A00EE66E500EE66EB6
:1022700071EC04F0E552E5520CD0360E01D0370E69
:10228000546F1200FE0EE66E30EC1EF0E55222ECAA
:1022900017F00101546B1200D9CFE6FFE1CFD9FF4F
:1022A000E652FD0EDB50030A08E0010A04E0030ACF
:1022B00006E1800E05D0C00E03D0940E01D0D40EDE
:1022C000DF6EFE0EDB04DF24E66E56EC1EF0E552F8
:1022D000E552E552E7CFD9FF1200D9CFE6FFE1CFB3
:1022E000D9FFFE0EDB50040A01E1E2D0070A01E14A
:1022F000A9D0010A71E0030A39E0010A01E00CD11A
:102300000101EC512AE0C72BC551030DF3CFE9FFC2
:10231000F4CFEAFFBF0EE926010EEA22020EE926FB
:10232000000EEA22EF50C75D09E3BF0EE66E010E14
:10233000E66EF6D8E552E55200090FE00101C551FD
:10234000030DF3CFE9FFF4CFEAFFBF0EE926010E3C
:10235000EA22EE52EF50C75D02E3000E01D0010EFB
:10236000E8B08280E8B0D8D08290D6D00101ED519B
:102370002AE0D02BCE51030DF3CFE9FFF4CFEAFFD3
:10238000C80EE926010EEA22020EE926000EEA2214
:10239000EF50D05D09E3C80EE66E010EE66EC0D8C0
:1023A000E552E55200090FE00101CE51030DF3CFD4
:1023B000E9FFF4CFEAFFC80EE926010EEA22EE5249
:1023C000EF50D05D02E3000E01D0010EE8B0828232
:1023D000E8B0A2D08292A0D00101EE512AE0D92B20
:1023E000D751030DF3CFE9FFF4CFEAFFD10EE92671
:1023F000010EEA22020EE926000EEA22EF50D95D14
:1024000009E3D10EE66E010EE66E8AD8E552E5527A
:1024100000090FE00101D751030DF3CFE9FFF4CF1D
:10242000EAFFD10EE926010EEA22EE52EF50D95D05
:1024300002E3000E01D0010EE8B08284E8B06CD057
:1024400082946AD00101EF512AE0E22BE051030DA2
:10245000F3CFE9FFF4CFEAFFDA0EE926010EEA2214
:10246000020EE926000EEA22EF50E25D09E3DA0EE1
:10247000E66E010EE66E54D8E552E55200090FE013
:102480000101E051030DF3CFE9FFF4CFEAFFDA0ECB
:10249000E926010EEA22EE52EF50E25D02E3000E61
:1024A00001D0010EE8B0828CE8B036D0829C34D0E6
:1024B0000101F0512AE0EB2BE951030DF3CFE9FFC5
:1024C000F4CFEAFFE30EE926010EEA22020EE92626
:1024D000000EEA22EF50EB5D09E3E30EE66E010E1B
:1024E000E66E1ED8E552E55200090FE00101E95100
:1024F000030DF3CFE9FFF4CFEAFFE30EE926010E67
:10250000EA22EE52EF50EB5D02E3000E01D0010E25
:10251000E8B0828EE8A0829EE552E7CFD9FF120094
:10252000D9CFE6FFE1CFD9FFFD0EDBCFE9FFFE0EED
:10253000DBCFEAFF080EE926000EEA22EF6AFD0E65
:10254000DBCFE9FFFE0EDBCFEAFF070EE926000E28
:10255000EA22EF2AEFCF00F0FD0EDBCFE9FFFE0EFF
:10256000DBCFEAFFE9CF01F0EACF02F0FD0EDBCFCF
:10257000E9FFFE0EDBCFEAFF060EE926000EEA2297
:10258000EF50030D0150F324E96E0250F420EA6E7F
:10259000EF50005C28E3FD0EDBCFE9FFFE0EDBCF42
:1025A000EAFF070EE926000EEA22EF6AFD0EDBCFF6
:1025B000E9FFFE0EDBCFEAFF060EE926000EEA2257
:1025C000EF5002E0000E01D0010EE66EFD0EDBCFF3
:1025D000E9FFFE0EDBCFEAFF060EE926000EEA2237
:1025E000E552E750EF6E010EE552E7CFD9FF12003A
:1025F000D9CFE6FFE1CFD9FFFC0EDBCFE9FFFD0E1F
:10260000DBCFEAFF060EE926000EEA22EF6AFC0E97
:10261000DBCFE9FFFD0EDBCFEAFF070EE926000E58
:10262000EA22EF6AFC0EDBCFE9FFFD0EDBCFEAFF0B
:10263000080EE926000EEA22EF6EFE0EDB50FD08C2
:1026400048E2FC0EDBCFE9FFFD0EDBCFEAFF030E15
:10265000E926000EEA22020EE926000EEA22EF68C1
:10266000FC0EDBCFE9FFFD0EDBCFEAFF030EE92610
:10267000000EEA22EF68FC0EDBCFE9FFFD0EDBCF98
:10268000EAFF030EE926000EEA22020EE926000EFA
:10269000EA22EF68FC0EDBCFE9FFFD0EDBCFEAFF9D
:1026A000020EE926000EEA22EF68FC0EDBCFE9FFFE
:1026B000FD0EDBCFEAFF030EE926000EEA22EE5202
:1026C000EF68FC0EDBCFE9FFFD0EDBCFEAFFEE5239
:1026D00050D0020EF36EFE0EDBCFF4FFF350F45C2D
:1026E0004BE2FC0EDBCFE9FFFD0EDBCFEAFF030E72
:1026F000E926000EEA22EE52EF6AFC0EDBCFE9FF7C
:10270000FD0EDBCFEAFFEE52000EEF6EFC0EDBCFCC
:10271000E9FFFD0EDBCFEAFF030EE926000EEA22F9
:10272000020EE926000EEA22EF68FC0EDBCFE9FF7D
:10273000FD0EDBCFEAFF030EE926000EEA22EF686A
:10274000FC0EDBCFE9FFFD0EDBCFEAFF030EE9262F
:10275000000EEA22020EE926000EEA22EF68FC0EC5
:10276000DBCFE9FFFD0EDBCFEAFF020EE926000E0C
:10277000EA22FF0EEF6E71D2FE0EDB507F0835E2CB
:10278000FE0EDB1CE76EFE0EE7CFDBFFDB50006EBC
:10279000016A3C683D6A416E01C042F00AEC1EF0DD
:1027A0003C50E66EFC0EDBCFE9FFFD0EDBCFEAFF0F
:1027B000EE52E552E750EF6EFF0FE66EFC0EDBCFF8
:1027C000E9FFFD0EDBCFEAFF030EE926000EEA2249
:1027D000EE52E552E750EF6EFC0EDBCFE9FFFD0E47
:1027E000DBCFEAFFEE52EF5022D0FC0EDBCFE9FF49
:1027F000FD0EDBCFEAFF030EE926000EEA22EE52C1
:10280000010EEF6EFC0EDBCFE9FFFD0EDBCFEAFF22
:10281000EE52010EEF6EFE0EDB50006E016A3C6858
:102820003D6A416E01C042F00AEC1EF03C50E66E7B
:10283000FC0EDBCFE9FFFD0EDBCFEAFF030EE9263E
:10284000000EEA22020EE926000EEA22E552E750C7
:10285000EF6EFC0EDBCFE9FFFD0EDBCFEAFF030ED0
:10286000E926000EEA22020EE926000EEA22EF28EF
:10287000E66EFC0EDBCFE9FFFD0EDBCFEAFF020EBA
:10288000E926000EEA22E552E750EF6EFE0EDBCF9E
:10289000E6FFFC0EDBCFE9FFFD0EDBCFEAFF020E09
:1028A000E926000EEA22EFCF04F0FC0EDBCFE9FFB1
:1028B000FD0EDBCFEAFF030EE926000EEA22020E30
:1028C000E926000EEA22EF50045C026E036AFE0E57
:1028D000DBCFE6FFFC0EDBCFE9FFFD0EDBCFEAFF2F
:1028E000030EE926000EEA22020EE926000EEA2275
:1028F000EF50E552E702F350006E016AFF0ED880F8
:102900000056000E015600C03CF001C03DF002C070
:1029100041F003C042F00AEC1EF03C50E66EFC0EA3
:10292000DBCFE9FFFD0EDBCFEAFFE552E750EF6EAC
:10293000E552E75CE66EFC0EDBCFE9FFFD0EDBCF78
:10294000EAFF030EE926000EEA22E552E750EF6E99
:10295000FC0EDBCFE9FFFD0EDBCFEAFFEF5001E11C
:1029600055D1FC0EDBCFE9FFFD0EDBCFEAFFEECF4A
:1029700000F0EECF01F0EFCF02F0030E036E426ED7
:1029800000C03DF0D3EC1FF0395001E0ACD0FC0E9C
:10299000DBCFE9FFFD0EDBCFEAFF030EE926000ED9
:1029A000EA22EECF04F0EECF05F0EFCF06F0030EF3
:1029B000076E426E04C03DF0D3EC1FF0395001E0C9
:1029C00092D0FC0EDBCFE9FFFD0EDBCFEAFFEECFAE
:1029D00000F0EECF01F0EFCF02F0330E036E426E47
:1029E00000C03DF0D3EC1FF039502BE1FC0EDBCFE3
:1029F000E9FFFD0EDBCFEAFF030EE926000EEA2217
:102A0000EECF04F0EECF05F0EFCF06F0330E076EF9
:102A1000426E04C03DF0D3EC1FF0395012E1330E8A
:102A2000006EFC0EDBCFE9FFFD0EDBCFEAFFEFCF40
:102A30003DF000C042F0D3EC1FF03DC0EFFF330E7D
:102A4000D1D0FC0EDBCFE9FFFD0EDBCFEAFFEECFEE
:102A500000F0EECF01F0EFCF02F00F0E036E426EEA
:102A600000C03DF0D3EC1FF039502BE1FC0EDBCF62
:102A7000E9FFFD0EDBCFEAFF030EE926000EEA2296
:102A8000EECF04F0EECF05F0EFCF06F00F0E076E9D
:102A9000426E04C03DF0D3EC1FF0395012E10F0E2E
:102AA000006EFC0EDBCFE9FFFD0EDBCFEAFFEFCFC0
:102AB0003DF000C042F0D3EC1FF03DC0EFFF0F0E21
:102AC00091D0030E006EFC0EDBCFE9FFFD0EDBCFD5
:102AD000EAFFEFCF3DF000C042F0D3EC1FF03DC065
:102AE000EFFF030E7FD0FC0EDBCFE9FFFD0EDBCF47
:102AF000EAFFEECF00F0EECF01F0EFCF02F0110EC3
:102B0000036E426E00C03DF0D3EC1FF039502BE154
:102B1000FC0EDBCFE9FFFD0EDBCFEAFF030EE9265B
:102B2000000EEA22EECF04F0EECF05F0EFCF06F074
:102B3000110E076E426E04C03DF0D3EC1FF0395009
:102B400012E1110E006EFC0EDBCFE9FFFD0EDBCFB4
:102B5000EAFFEFCF3DF000C042F0D3EC1FF03DC0E4
:102B6000EFFF110E3FD0FC0EDBCFE9FFFD0EDBCFF8
:102B7000EAFFEECF00F0EECF01F0EFCF02F0050E4E
:102B8000036E426E00C03DF0D3EC1FF0395065E19A
:102B9000FC0EDBCFE9FFFD0EDBCFEAFF030EE926DB
:102BA000000EEA22EECF04F0EECF05F0EFCF06F0F4
:102BB000050E076E426E04C03DF0D3EC1FF0395095
:102BC0004CE1050E006EFC0EDBCFE9FFFD0EDBCF06
:102BD000EAFFEFCF3DF000C042F0D3EC1FF03DC064
:102BE000EFFF050E006EFC0EDBCFE9FFFD0EDBCF25
:102BF000EAFF030EE926000EEA22EFCF3DF000C007
:102C000042F0D3EC1FF03DC0EFFF27D0FC0EDBCF2E
:102C1000E9FFFD0EDBCFEAFF030EE926000EEA22F4
:102C2000EF68FC0EDBCFE9FFFD0EDBCFEAFF030E02
:102C3000E926000EEA22EECF00F0EECF01F0EFCF52
:102C400002F0FC0EDBCFE9FFFD0EDBCFEAFF00C098
:102C5000EEFF01C0EEFF02C0EEFFE552E7CFD9FF65
:102C60001200FF001200D9CFE6FFE1CFD9FF060E18
:102C7000E12644EC1FF00009FCE1010EE66E56EC83
:102C80001EF0E55244EC1FF00009FCE10C0EE66E6C
:102C900056EC1EF0E552E8EC1FF0AC0EE66E010EAD
:102CA000E66E020EE66EE66A29EC1FF0E552E5528A
:102CB000E66E9EDCE552E552E552B50EE66E010E7B
:102CC000E66E030EE66EE66A29EC1FF0E552E55269
:102CD000006E016AFF0ED8800056000E0156020EEB
:102CE000416E426A00C03CF001C03DF00AEC1EF0AB
:102CF0003CC000F03DC001F03C50E66E79DCE5528E
:102D0000E552E55244EC1FF00009FCE1010EE66ECD
:102D1000E66E4CEC11F0E552E5527A0EDE6E3F0E97
:102D2000DD6E0E0EF36E020EF3CFDBFF030EDB6AD9
:102D3000040EDB6A050EDB6A040EDBCF00F0050E25
:102D4000DBCF01F0020EDBCF02F0030EDBCF03F08E
:102D50000250005C035001581CE244EC1FF00009D3
:102D6000FCE1040EDBCF00F0050EDBCF01F0DE50FE
:102D70000024F66EDD500120F76E0800F550E66E77
:102D800030EC1EF0E552040EDB2A050ED5E3DB2AFB
:102D9000D3D744EC1FF00009FCE1020EE66E010EF1
:102DA000E66E4CEC11F0E552E5526C0EDE6E3F0E15
:102DB000DD6E0D0EF36E020EF3CFDBFF030EDB6A4A
:102DC000040EDB6A050EDB6A040EDBCF00F0050E95
:102DD000DBCF01F0020EDBCF02F0030EDBCF03F0FE
:102DE0000250005C035001581CE244EC1FF0000943
:102DF000FCE1040EDBCF00F0050EDBCF01F0DE506E
:102E00000024F66EDD500120F76E0800F550E66EE6
:102E100030EC1EF0E552040EDB2A050ED5E3DB2A6A
:102E2000D3D70101040EAB6FA76BF28E010EA96F11
:102E3000060EE15C02E2E16AE552E16EE552E7CF9F
:102E4000D9FF1200E8EC1FF0E668FF0EE66EE66AB6
:0E2E5000A2EC1EF0E552E552E55233EF16F00B
:022E5E006C50B6
:102E60000CE16896040100513C0BE842E8420D0871
:102E700002E10AD8010C41D8010C040E6C5C03E19C
:102E800068964AD8010C000CD9CFE6FFE1CFD9FFF4
:102E9000E652040104BF046B0001806B786B796B10
:102EA0007E6B7F6B98EC1AF0DF6ADF50006E016A70
:102EB000010E005C000E01581AE20001795117E181
:102EC000F76ADF34FE0BF736F66EA10EF6263B0EE0
:102ED000F7220900F5CF00F00800F5CF01F004D08B
:102EE00001C0FAFF0050F96EFBDFDF2ADED7E8D819
:102EF000E552E552E7CFD9FF1200020E0001785DDE
:102F000009E1A1D8040100BD02D0C80E01D0880E8D
:102F1000006F1200A5EF18F0040E0101FC5D09E13D
:102F200022C46EFF6E50000802E2050E01D0030EAF
:102F3000FC6F0001780510E111D8020E0001805DE0
:102F400003E10401840E06D0040104BD02D0C80EC2
:102F500001D0880E046F1200A5EF18F0D9CFE6FF5C
:102F6000E1CFD9FF020EE1260001080E7E5D000EC2
:102F70007F590DE27EC0DEFF7FC0DDFF805102E1A0
:102F8000010E03D0800506E1020E806F03D0080E0B
:102F9000DE6EDD6A040104930491010EDB5004131C
:102FA000DFCF05F4000EDB5000017E5F010EDB5029
:102FB0007F5B280E7C6F040E7D6F0101FDA31DD089
:102FC000D9CFE9FFDACFEAFFEE50ED1032E07AC058
:102FD000F6FF7BC0F7FF0800F5507CC0E9FF7DC01D
:102FE000EAFFEF6E00017C2B000E7D237A2B7B2302
:102FF000DF06010EE5E2DB06E3D7D9CFE9FFDACF42
:10300000EAFFEE50ED1015E07AC0E9FF7BC0EAFF61
:10301000EF507CC0E9FF7DC0EAFFEF6E00017C2B22
:10302000000E7D237A2B7B23DF06010EE6E2DB0612
:10303000E4D7020EE15C02E2E16AE552E16EE5529C
:10304000E7CFD9FF1200D9CFE6FFE1CFD9FF020EBB
:10305000E126030E04010015E76E010EE7CFDBFF4A
:1030600001C4DFFFDE5000017E27DD507F23280EE4
:103070007A6F040E7B6FD9CFE9FFDACFEAFFEE500B
:10308000ED1014E07AC0E9FF7BC0EAFFEF507CC08E
:10309000E9FF7DC0EAFFEF6E7C2B000E7D237A2BCB
:1030A0007B23DF06010EE7E2DB06E5D7020EE15CDB
:1030B00002E2E16AE552E16EE552E7CFD9FF120084
:1030C0006D98000179510BE10401080E016F200E8B
:1030D000026F040E036F840E006F040123D00401FD
:1030E00020AF22D000017E510401265D00017F51F6
:1030F0000401275904E226C47EF027C47FF02EDFA6
:103100000001010E786F0401080E016F200E026F9E
:10311000040E036F800E006F0401280E066F040E6C
:10312000076FC80E046F12000001020E786F0401D1
:10313000056BC80E046F0401080E016F280E026FA4
:10314000040E036FC80E006F1200D9CFE6FFE1CF67
:10315000D9FFE652020E0001785D35E16D50100B8B
:1031600032E004010151006E016A080E00182BE1E3
:10317000015029E100513C0BE842E8420D0823E1EF
:103180000051800B20E1200E026F040E036FDF6AF6
:10319000DF50006E016A080E005C000E015820E24C
:1031A000DF50EA6A280FE96E040EEA22EF50E66E5D
:1031B000DF50EA6A200FE96E040EEA22E552E7507A
:1031C000EF6EDF2AE5D70001786B0401080E016F6E
:1031D000200E026F040E036F8C0E006F0401046B4F
:0A31E000E552E552E7CFD9FF1200D7
:0631EA00040120511F0B3F
:1031F000010801E012002051600BE842E842E84279
:10320000E842E842010801E01200245103E02405ED
:1032100001E012002151230A43E0010A3BE0030AC6
:103220002BE0010A20E0240A3BE0070A39E0010A0A
:1032300037E0030A10E0010A01E012000001030E6A
:10324000796F0001700E7A6F000E7B6F0101FD93A4
:103250000001080E1DD00001030E796F0001700EF1
:103260007C6F000E07D00001030E796F0001680E1D
:103270007C6F000E7D6F12000001030E796F00015C
:10328000680E7A6F000E7B6F0101FD930001070E3F
:103290007E6F12000001030E796F22C46FF01200DE
:1032A00012000001686BC20E696F010E6A6F6B6BD2
:1032B0006C6B6D6B080E6E6F616B606B1A0E726ECD
:1032C0001E0E736E0401300E166F040E176F400E43
:1032D000146F0401196F380E1A6F040E1B6F880EDD
:1032E000186F0401780E1E6F040E1F6F400E1C6FC6
:1032F0001200D9CFE6FFE1CFD9FF0001606B0401D6
:1033000018BF30D0FC0EDBCF00F01951D88000542C
:1033100003E2FC0E19C4DBFF0001606BFC0EDB5006
:10332000605D19E26051EA6A380FE96E040EEA2224
:10333000EF50E66E6051E76EFD0EDBCFE9FFFE0E4B
:10334000DBCFEAFFE750E926000EEA22E552E7501C
:10335000EF6E602BE3D70401400E196F1817187D2C
:10336000880E181300016051E552E7CFD9FF120013
:10337000D9CFE6FFE1CFD9FFE6520001615129E143
:10338000DF6ADF2AFF0EDF5C0BE0FD0EDBCFE9FF1B
:10339000DB2AFE0EDBCFEAFF01E3DB2AEF50F1E18F
:1033A000DF50006E016AD950FD0FE96EFF0EDA2082
:1033B000EA6E0050EE5E0150ED5AFD0EDBCF62F07A
:1033C000FE0EDBCF63F0DFCF66F00001676B010E0E
:1033D000616FE552E552E7CFD9FF1200D9CFE6FF82
:1033E000E1CFD9FFE652000161512AE1DF6ADF2A0D
:1033F000FF0EDF5C0CE0FD0EDBCFF6FFDB2AFE0EDE
:10340000DBCFF7FF01E3DB2A0800F550F0E1DF50E6
:10341000006E016AD950FD0FE96EFF0EDA20EA6EE8
:103420000050EE5E0150ED5AFD0EDBCF62F0FE0E55
:10343000DBCF63F0DFCF66F00001010E676F616FD5
:10344000E552E552E7CFD9FF1200D9CFE6FFE1CF31
:10345000D9FFE65204011CBF66D0030E0001615D76
:1034600001E1616B61515FE0020E615D03E1040106
:103470001D6B50D0610551E1400E006E016A66512E
:10348000005C000E015803E2400EDF6E02D066C001
:10349000DFFFDFCF1DF4DF50665D666F780E646F6F
:1034A000040E656F670514E1DF5025E062C0F6FF8A
:1034B00063C0F7FF0800F55064C0E9FF65C0EAFF8C
:1034C000EF6E642B000E6523622B6323DF06ECD7BF
:1034D000DF5011E062C0E9FF63C0EAFFEF5064C053
:1034E000E9FF65C0EAFFEF6E642B000E6523622BD7
:1034F0006323DF06EDD7000166510FE104011D5182
:10350000006E016A400E001805E1015003E1000160
:10351000020E02D00001030E616F400E04011C1761
:103520001C7D880E1C13E552E552E7CFD9FF12002F
:1035300004012051600BE842E842E842E842E842D8
:10354000000901E012002151070A4CE00B0A4AE091
:10355000070A3BE0010A27E00B0A23E0020A21E008
:10356000030A1DE0080A12E0010A0EE00F0A0AE051
:10357000030A01E012000001010E796F0101040E3F
:10358000FC6F1200F3EF1AF04AEF1BF00001010E7E
:10359000796F0001FE0E7A6F010E7B6F10D071EF14
:1035A0001BF0BCEF1BF00001010E796F04012451E8
:1035B00000017A6F7B6BFF0E7A27010E7B230101DE
:1035C000FD930001010E7E6F12000001010E796F64
:1035D00004012451EA6AFF0FE96E010EEA2222C4B7
:1035E000EFFF12001200800E0401205D52E1235112
:1035F000030A30E0010A0CE0030A49E10001010E70
:10360000796F00011C0E7A6F3B0E7B6F120E3CD05F
:103610000001010E796F04012251F66EF76AD8900D
:10362000F636F736970EF6263B0EF7220900F5CF51
:103630007AF00A00F5CF7BF0020E0001F76A7A25D6
:10364000F66E7B51F7220900F5CF7EF00A00F5CF28
:103650007FF01DD00001010E796F04012251F66E3A
:10366000F76AD890F636F7369B0EF6263B0EF72211
:103670000900F5CF7AF00A00F5CF7BF07AC0F6FFAB
:103680007BC0F7FF0800F55000017E6F7F6B0101E2
:10369000FD8312000001010E796F0F0EE66E710EB0
:1036A000E66E0F0EE66ECBEC1CF0E552E552E552ED
:1036B000010EE66EFF0EE66E010EE66ECBEC1CF020
:1036C000E552E552E55222C4FEF10401225104E123
:1036D0000101050EFC6F12000101060EFC6F51EF97
:1036E00019F00401286B296B040120511F0B020AF9
:1036F00013E0030A0DE0010A31E10001010E796FC8
:10370000040128810101FDA129D00401288326D0CC
:103710000001010E796F22D00001010E796F0401C2
:1037200024510F0B080DF350016A000F006E040EB8
:1037300001222451800B01E0010E040DF350000121
:1037400000247C6F000E01207D6F7CC0E9FFEA6ED3
:10375000EF50040B03E00401010E286F000179050E
:103760000AE10001280E7A6F040E7B6F0101FD93C0
:103770000001020E7E6F12000401220510E12051AB
:103780001F0B00090CE10001010E796F030E04010B
:10379000215D03E10101FD8102D00101FD910401E0
:1037A000225136E120511F0B020832E124510F0B48
:1037B00000092EE00001010E796F040124510F0B66
:1037C000080DF350016A000F006E040E012224510F
:1037D000800B01E0010E040DF350000100247C6F0A
:1037E000000E01207D6F030E0401215D02E1840EB5
:1037F00003D024AF07D0400E7CC0E9FF7DC0EAFFB4
:10380000EF6E1200880E7CC0E9FF7DC0EAFFEF6E0C
:023810001200A4
:0E3812006DA60CD80101FC0508E16DBA06D0C8
:10382000686A696A69806988020EFC6F12006D6AB5
:10383000696A6D860101010EFC6F12006D6A696A8A
:103840000101FC6B12001EEF1CF00101FC5101E1B3
:1038500012006850040B04E06950040B01E046D8E4
:103860006DB212006850010B04E06950010B01E0D9
:103870006AD86850100B04E06950100B01E02ED894
:103880006850400B04E06950400B01E048D8685094
:10389000200B04E06950200B01E043D86850020B74
:1038A00004E06950020B01E04CD8030E0101FC5DFD
:1038B00001E212000001816B040E815D0EE268508E
:1038C000080B0BE06950080B08E02FEC17F000091B
:1038D00001E168960001812BEFD712006984689896
:1038E0006D82A19AA08A0300A09A12006D92699439
:1038F00068A402D06894FCD712000101FDA10ED08B
:103900006D926D840001080E826F070E836F82072F
:10391000000E835B82518311FAE16D941200689C62
:10392000120070A00CD0800E0401005D07E1840E2F
:103930000401045D03E104018C0E006F7090689A2D
:1039400012006A6A12006A6A686A9F0E6B6E7B0ECA
:10395000696E6E6A0F0EE66E710EE66E0F0EE66E03
:103960001AD8E552E552E552160E706E68A608D0D8
:103970006896000000000000000000000000F6D77C
:103980006D98A5EC18F00101FD910101FE6B01019C
:10399000030EFC6F1200D9CFE6FFE1CFD9FFFD0E79
:1039A000DBCFE9FFFE0EDBCFEAFFFC0EDB5004E0CD
:1039B000EE6AFC0EDB06F9D7E552E7CFD9FF12001D
:1039C0000F0E8116F00E9312939493929396819416
:1039D000819281961200D9CFE6FFE1CFD9FF1DEC8D
:1039E00004F00F0E93168116818A818616EC04F07E
:1039F000819623EC04F00F0E8116818A818616ECE5
:103A000004F0819629EC04F00F0E8116818A8186DC
:103A100016EC04F08196F00E931244EC1FF00009AE
:103A2000FCE1FE0EDBCFE6FF56EC1EF0E55244EC67
:103A30001FF00009FCE1080EE66E56EC1EF0E552A0
:103A400044EC1FF00009FCE1010EE66E56EC1EF09E
:103A5000E55244EC1FF00009FCE1060EE66E56EC60
:103A60001EF0E55244EC1FF00009FCE1800EE66E0A
:0E3A700056EC1EF0E552E552E7CFD9FF1200EA
:023A7E002A0E0E
:103A8000F66E080EF76E000EF86E01010900F55093
:103A9000F76F0900F550F86F03E1F76701D03DD0EB
:103AA0000900F550F26F0900F550F36F0900F55069
:103AB000F46F09000900F550E96E0900F550EA6E4F
:103AC000090009000900F550F56F0900F550F66F7F
:103AD00009000900F6CFF9F1F7CFFAF1F8CFFBF1C1
:103AE000F2C1F6FFF3C1F7FFF4C1F8FF0101F5538E
:103AF00002E1F65307E00900F550EE6EF507F8E233
:103B0000F607F9D7F9C1F6FFFAC1F7FFFBC1F8FFD5
:0C3B10000101F707000EF85BBFD71200A0
:043B1C001201000290
:103B200002000008CD5BCD5B01000102000109022B
:103B30004300020100A07D0904000001020201000F
:103B400005240010010424020205240600010524B6
:103B50000100010705820308000209040100020AAE
:103B60000000000705030240000007058302400033
:103B70000004030904100355005300420032004CB6
:103B80000043004400120355005300420032004C31
:103B900000430044002B002E3B2E3B713B753B85C0
:033BA0003BEA31CC
:0C3BA4003A503F02F3CF36F0F4CF37F078
:103BB0004002F3503726000EF420386E3A5041028E
:103BC000F3503826000EF420396E3A504202F3507A
:103BD00039263B503F02F3503726F4503822000E6E
:103BE00039223B504002F3503826F45039223B50E2
:103BF0004102F35039263C503F02F3503826F4502E
:103C000039223C504002F35039263D503F02F350D8
:043C1000392612003F
:0C3C1400346A42AE13EF1EF0416C421EF9
:103C2000E86A4222341E3DAE1BEF1EF03C6C3D1E86
:103C3000E86A3D22341E90EC1FF03DBE2BEF1EF0D3
:103C400034AE000C3C6C3D1EE86A3D22386C391ED7
:103C5000E86A3922000C34BE22EF1EF03588FF0CD2
:103C6000D9CFE6FFE1CFD9FF0F0E93168116FE0ED6
:103C7000DB50F00B81128182819416EC04F0818676
:103C800016EC04F081960F0E8116FE0EDB38F00B59
:103C9000F00B811216EC04F0818616EC04F081968C
:0C3CA000F00E9312E552E7CFD9FF12009E
:043CAC00D9CFE6FF87
:103CB000E1CFD9FF0F0E93168116FE0EDB50F00BED
:103CC00081128194819216EC04F0818616EC04F046
:103CD00081960F0E8116FE0EDB38F00BF00B811271
:103CE00016EC04F0818616EC04F08196F00E931227
:083CF000E552E7CFD9FF1200F5
:083CF800DACFE4FFE652F2A46A
:103D000004D0F2940101A72B01D0F26AE552E5CF6D
:103D1000DAFF1100D8CFE4FFE0CFE4FFE46EDACFA2
:103D2000E4FFE652F2A404D0F2940101A72B01D0E3
:103D3000F26AE552E5CFDAFFE550E5CFE0FFE5CFE7
:043D4000D8FF100098
:0C3D4400D9CFE6FFDACFE6FFE1CFD9FFD0
:103D5000E2CFDAFFFF0EE76EFC0EDBCF00F0E7509C
:103D600000160050A96EFB0EDB50A86EA69EA69C06
:103D7000A684F29E550EA76EAA0EA76EA682F28E9C
:0E3D8000A694E552E5CFDAFFE7CFD9FF120097
:023D8E00396A90
:103D9000386A376A366A200EE76ED8903A363B3674
:103DA0003C363D3636363736383639363F50365C57
:103DB00040503758415038584250395809E33F5025
:103DC000365E4050375A4150385A4250395A3A2A92
:063DD000E72EE4D712000B
:0A3DD600D9CFE6FFE1CFD9FFE65296
:103DE0008184818216EC04F0818616EC04F0F00EDA
:103DF0008114DF6E819616EC04F0818616EC04F0D7
:103E000081380F0B0F0BDF12819681928194DF5066
:0A3E1000E552E552E7CFD9FF12009A
:063E1A00D9CFE6FFDACF6C
:103E2000E6FFE1CFD9FFE2CFDAFFFD0EDB507F0BDB
:103E3000D56ED76AD66AF294FD0EDBAE02D0F28A56
:103E400001D0F29AD58EE552E5CFDAFFE7CFD9FF60
:023E500012005E
:0E3E5200D9CFE6FFDACFE6FFE1CFD9FFE2CF0E
:103E6000DAFFFF0EE76EFC0EDBCF00F0E750001626
:103E70000050A96EA69CA69EA680A850E552E5CF4C
:083E8000DAFFE7CFD9FF1200C1
:083E88008184819216EC04F024
:103E9000818616EC04F081AE09D0819616EC04F010
:103EA000818616EC04F081968194010C819616ECC3
:0E3EB00004F0818616EC04F081968194000CDB
:023EBE0007D823
:103EC00010D8CDEC04F00DD8D3EC04F0FCD7140ED0
:103ED0006F6E0101FC6B0101FD6B0101FE6BA1EF37
:103EE00004F009EC1CF06FBE02D025EC1CF025EFAD
:023EF0001AF0C6
:0E3EF200FF0EE350456EEF0E01D0F30EE76EAB
:103F0000E72E80EF1FF00C0E446EE76AE72E86EF77
:103F10001FF0442E85EF1FF0452E7EEF1FF012009C
:103F2000396A386A100EE76ED8903C363D3638361E
:103F300039364150385C4250395805E34150385EBB
:0C3F40004250395A3C2AE72EF0D71200FC
:043F4C00FF0EE35031
:103F5000456E480E01D04C0EE76EE72EFED7E76A9D
:0C3F6000E72EFED7452EF7D70000120018
:043F6C00446F206E10
:103F70006F7420756E706C7567005265736574742C
:093F8000696E6720696E203300B0
:063F8A0013EE00F023EE2F
:103F900000F0F86A359C3FEC1DF0EBEC1FF05FEC95
:063FA0001FF0FBD7120028
:0A3FA600396A080EE76ED8903D3628
:103FB00039364250395C02E3396E3D2AE72EF7D795
:023FC0001200ED
:0E3FC20000EE00F00F0EEE6AEA62FDD712006C
:063FD000A6B2FED71200AC
:023FD6001200D7
:00000001FF
